:1000000000308A0090280000FF00030E8301A10049
:100010000A08A0008A010408A2007708A300780853
:10002000A4007908A5007A08A6007B08A70083131E
:1000300083128C308400001C1F280C1832282208E0
:1000400084002308F7002408F8002508F900260892
:10005000FA002708FB0020088A00210E8300FF0E0B
:100060007F0E09008A110A1246280A108A100A1106
:100070008207403406345B344F3466346D347D344B
:1000800007347F346F348034003440340030A802A9
:10009000031C0130A9020130031C0230AA02003007
:1000A000031C0130AB02AB08031D69282A08003C81
:1000B000031C69288030A807843003188530A907FD
:1000C0001E3003181F30AA07003003180130AB0799
:1000D000AC0A0C108A110A121F28AB011E30AA00AC
:1000E0008430A9008030A8000530900083160C14DD
:1000F00083128A110A121F293430840083130008E6
:1001000003198F280230F800F701F70B8528F80B48
:1001100084289730F700F70B8B28800B8228003457
:1001200003081F3983005730F70020308400831301
:100130008001840AF70B9828F801F901FA01FB0104
:10014000FC01FD01FE015030F700A0308400831354
:100150008001840AF70BA8286030F7001030840073
:1001600083178001840AF70BB12883136030F700EE
:100170009030840083178001840AF70BBB28831317
:10018000A001840183131F308305713083168F0013
:100190000F0803170908C039890003131F129F12A3
:1001A0000030031788008312870188018901031337
:1001B000AC01AD01AE01AF01B001FF30B20083165A
:1001C00003170908C039890003131F129F1200305A
:1001D00003178800831203131F109412B2123208FF
:1001E0008316870083123216320883168700831223
:1001F000B211320883168700013083129400003058
:10020000831694000108C739083881000030F800CF
:100210008312920000308316920083120317870125
:10022000880189017130831603138F000F08053090
:100230008312850000308316850083126D28AC017F
:100240002E083520F8008500B21432088316870086
:10025000831287185229AE01AF012E083520F8000D
:100260008500B215320883168700831232163208D1
:10027000831687008312B216320883168700831212
:1002800032173208831687008312B217320883169A
:10029000870001308312B000AC0183160C14C0300B
:1002A00083128B04300BC92BFF3083168600831218
:1002B0000608B1003108FE3A03197429033A0319FC
:1002C0007729063A03197A290C3A03197D29183A35
:1002D00003198029303A03198329603A03198629C2
:1002E000C03A031989298C290130AE008E290230C9
:1002F000AE008E290330AE008E290430AE008E2968
:100300000530AE008E290630AE008E290730AE00D3
:100310008E290830AE008E29AE018E29AE08031D4D
:10032000AA29B215320883168700831232163208C2
:10033000831687008312B216320883168700831251
:1003400032173208831687008312B21732088316D9
:10035000870083122E0BED2983160C1083120B13CA
:100360008B138B1BB0292E083520F8008500B001B7
:10037000B2113208831687008312871532163208AD
:10038000831687008312B216320883168700831201
:1003900032173208831687008312B213320883168D
:1003A0008700831287130130AF002F08033C031C22
:1003B000ED293210320883168700831207141E308D
:1003C000B4007C2032103208831687008312071095
:1003D0001E30B4007C20AF0AD5292E08023C031D34
:1003E000312A83160C1083120B138B138B1BF529E8
:1003F0002E083520F8008500B001B21532088316AA
:100400008700831232123208831687008312071680
:10041000B216320883168700831232173208831609
:1004200087008312B2133208831687008312871362
:10043000AF012F08033C031C312A32103208831607
:100440008700831207141E30B4007C20321032085B
:1004500083168700831207101E30B4007C20AF0A79
:10046000192A2E08033C031D752A83160C108312CB
:100470000B138B138B1B392A2E083520F8008500AF
:10048000B001B21532088316870083123216320883
:10049000831687008312B2123208831687008312F4
:1004A000871632173208831687008312B213320878
:1004B0008316870083128713AF012F08033C031CA8
:1004C000752A3210320883168700831207141E30F3
:1004D000B4007C2032103208831687008312071084
:1004E0001E30B4007C20AF0A5D2A2E08043C031D98
:1004F000B92A83160C1083120B138B138B1B7D2AC6
:100500002E083520F8008500B001B2153208831698
:100510008700831232163208831687008312B216C0
:10052000320883168700831232133208831687003D
:1005300083120717B21332088316870083128713BA
:10054000AF012F08033C031CB92A3210320883166E
:100550008700831207141E30B4007C20321032084A
:1005600083168700831207101E30B4007C20AF0A68
:10057000A12A2E08053C031DFD2A83160C108312A8
:100580000B138B138B1BC12A2E083520F800850016
:10059000B001B21132088316870083128711321618
:1005A0003208831687008312B2163208831687003A
:1005B000831232173208831687008312B21332086F
:1005C0008316870083128717AF012F08033C031C93
:1005D000FD2A3210320883168700831207141E305A
:1005E000B4007C2032103208831687008312071073
:1005F0001E30B4007C20AF0AE52A2E08063C031DFD
:10060000412B83160C1083120B138B138B1B052BA2
:100610002E083520F8008500B001B2153208831687
:100620008700831232123208831687008312071262
:10063000B2163208831687008312321732088316E7
:1006400087008312B213320883168700831287173C
:10065000AF012F08033C031C412B321032088316D4
:100660008700831207141E30B4007C203210320839
:1006700083168700831207101E30B4007C20AF0A57
:10068000292B2E08073C031D852B83160C10831283
:100690000B138B138B1B492B2E083520F80085007C
:1006A000B001B21532088316870083123216320861
:1006B000831687008312B2123208831687008312D2
:1006C000871232173208831687008312B21332085A
:1006D0008316870083128717AF012F08033C031C82
:1006E000852B3210320883168700831207141E30C0
:1006F000B4007C2032103208831687008312071062
:100700001E30B4007C20AF0A6D2B2E08083C031D60
:10071000C92B83160C1083120B138B138B1B8D2B81
:100720002E083520F8008500B001B2153208831676
:100730008700831232163208831687008312B2169E
:10074000320883168700831232133208831687001B
:1007500083120713B2133208831687008312871798
:10076000AF012F08033C031CC92B3210320883163B
:100770008700831207141E30B4007C203210320828
:1007800083168700831207101E30B4007C20AF0A46
:10079000B12BB008031DE72BAE080319E72B14306B
:1007A000B300FA30B4007C20B30BD12B32103208E6
:1007B00083168700831207146430B4007C20321043
:1007C000320883168700831207100130B0002C080E
:1007D000053C031D0A2CAE08031D0A2C83160C10C1
:1007E00083120B138B138B1BF22BB001AC01321055
:1007F000320883168700831207140430B300C83010
:10080000B4007C20B30BFF2B321032088316870014
:10081000831207102D082C0203191B2C32153208E5
:10082000831687008312071D1B2C2C08AD002C0893
:100830003520F80085002D082C0203192C2C3215C8
:10084000320883168700831207192C2C2C08AD0060
:0C0850002E083520F800850024296300E4
:04400E009423FF3FB9
:00000001FF
